:020000040000fa
:080000001406040000000000da
:020000040000fa
:020000040002f8
:04afe000dfff00008f
:020000040000fa
:020000040002f8
:04afe400ffff00006b
:020000040000fa
:020000040002f8
:04afe80078ff0000ee
:020000040000fa
:020000040002f8
:04afec007dff0000e5
:020000040000fa
:020000040002f8
:04aff00078ff0000e6
:020000040000fa
:1000080000000000000000000000000000000000e8
:100018000c060000000000000000000000000000c6
:10002800000000000000000000000000b00900000f
:1000380000000000000000000000000000000000b8
:10004800f20900000000000000000000bc0a0000e7
:10005800280b0000540b0000000000000000000006
:100068000000000000000000000000000000000088
:100078000000000000000000000000000000000078
:10008800000000000000000000000000380a000026
:100098007a0a0000000000000000000000000000d4
:1000a8000000000000000000000000000000000048
:1000b8000000000000000000000000000000000038
:1000c8000000000000000000000000000000000028
:1000d8000000000000000000000000000000000018
:1000e8000000000000000000000000000000000008
:1000f80000000000000000000000000000000000f8
:1001080000000000000000000000000000000000e7
:1001180000000000000000000000000000000000d7
:1001280000000000f40a00000000000000000000c9
:1001380000000000000000000000000000000000b7
:1001480000000000000000000000000000000000a7
:100158000000000000000000000000000000000097
:100168000000000000000000000000000000000087
:100178000000000000000000000000000000000077
:100188000000000000000000000000000000000067
:100198000000000000000000800b0000ac0b000015
:1001a800d80b000000000000000000000000000064
:1001b8000000000000000000000000000000000037
:1001c8000000000000000000000000000000000027
:1001d8000000000000000000000000000000000017
:1001e8000000000000000000000000000000000007
:1001f80000000000000000000000000000000000f7
:1002080000000000000000000000000000000000e6
:1002180000000000000000000000000000000000d6
:1002280000000000000000000000000000000000c6
:1002380000000000000000000000000000000000b6
:1002480000000000000000000000000000000000a6
:100258000000000000000000000000000000000096
:100268000000000000000000000000000000000086
:0c0278000000000000000000000000007a
:020000040000fa
:1004000027d2bf002652b7004220af002672ec0070
:1004100027d2d60027d2b60000c0d20027d2bf0014
:1004200000c0fd0027f2b70026d2bf0000c0fd00cb
:100430000040d20027d2b60027d2bf0000c0fd0086
:1004400027f2b7001040b20026f2d60026f2b6001e
:1004500027f2d6003091800000000600803e200088
:10046000030007008100e900fcff3a0000000600dd
:10047000831f7800c20320000400bc006601510005
:10048000e0815900f23fb1000380b1000600350061
:10049000ee03090000000000423fb1000380b100fc
:1004a000fbff3d001200b000223fb000020035000b
:1004b0000280090000000000cf0178000000060063
:1004c000889fbe008a9fbe008c1f78000004be007b
:1004d000850107000478a30026003a006120e100ae
:1004e0002500320009f8a30025003a006420e1004d
:1004f00021003200f507b1000508a3000200320018
:1005000000004000818048006044b80003102000d3
:1005100002002000000040008180480008054400df
:1005200089854c000a0541008b8549000a05500069
:100530008b855800030033000a00be0002047400db
:10054000838474008301d1000281d300830f710082
:10055000f0ff3a008904d1000884d300600149000b
:1005600082017800c1adde00fb07b0007301070017
:10057000070037000960a0000800be000400370033
:100580001202200062918800f0ff2f00f1ff270087
:100590004f0678004f05be004f04be000000060065
:1005a00003f0a200869fbe00889fbe008a9fbe0007
:1005b0008c9fbe0044010700860133006450e100b7
:1005c0004f0032006420e1005200320003826c00d0
:1005d00007003b000905d0000306d000820f54003d
:1005e0000c065d000200390002003200890178002b
:1005f000030678008582550004003d000003fd00dd
:100600008103fd008502ea008b854200840f7200a1
:1006100002003b0060001000e08018006011b8008c
:100620000005eb007a28e1000a0039000600780096
:10063000c75ddd00f707b200878075002d00370029
:10064000828171000a017800610560008180d1001b
:100650000080d3008502e900f9ff3b00060440005a
:100660008784480002003b0060041400e0841c0002
:100670000988a300070032008a817100828171001d
:10068000610164008904d1000884d3008b05e8006f
:10069000170037000978a30013003a000b00e000b0
:1006a000130034008b05e9000804440089844c00e1
:1006b0000a4474000978a3000d003a000b00e00022
:1006c000070034008b05e9000804440089844c00cd
:1006d00001003a000b0020000978a300f7ff320068
:1006e0000001eb0002003700828171000a017800ee
:1006f000120107000cf0a70001f0a0003e01370036
:100700006420e10002003a00838f6c003f01330057
:100710000801be000200be0037013700869fbe0000
:10072000889fbe008a9fbe008c9fbe00e600070027
:100730002801330003866c006450e1002e00320073
:100740006420e100330032006150e1002f003200ec
:100750006120e1003100320085855500eb07b000d3
:1007600009002000080420000500370008044400a8
:1007700089844c000a0031000603430087834b0044
:100780000001530081815b00f8ff33000203be00cb
:100790000800a0000804440089844c00f6ff3900da
:1007a000c639dd0083017300010032001300200010
:1007b0008904d1000884d3000998a3000500320001
:1007c0000800a7000300a0008904d1000884d3001a
:1007d0008b05e8008904d1000884d3000001eb00f8
:1007e0000281d200d500070001f0a1000cf0a700a3
:1007f00001f0a000000137006420e1000301320095
:100800000801be000200be00f7ff37006120e100d2
:10081000fe0032006000b800f3ff37000000200047
:1008200001f82700f0ff3700869fbe00889fbe00ba
:100830008a9fbe008c9fbe00a3000700e500330026
:1008400003866c006450e100240032006420e10063
:10085000270032006150e100220032006120e100f7
:10086000210032008b854200eb07b1000134b80053
:10087000003ab8000804420089844a00013ab800ee
:100880000030b8008880400009014a0004003300ad
:100890000000400081804800020149008b05e9000a
:1008a000c909dd008301700001003200130020003f
:1008b000c814de004814dd004709de001200b20053
:1008c000c808de00088470009c00070001f0a10049
:1008d0000cf0a70001f0a000c70037006120e10084
:1008e000ca0032000801be000200be00f7ff370058
:1008f0006150e100fcff3a00c4003700829fbe0057
:100900000001be00780007000470a70003f0a100fa
:100910006509b100180032000e0035006828e100ba
:1009200007003500f0ff2f00f1ff27000300e00073
:1009300015003b00010028004f01be00000005002b
:1009400000004000818048008502e900fcff3a0079
:1009500009003700f88f420003003c008000eb00e4
:100960004f01be00000005008100d1000080d300cf
:100970008502e800fcff3a000300e00002003b00b3
:1009800060001000e08018004f01be00000006006b
:10099000829fbe000001be00530007000470a70044
:1009a00003f0a10003f8a30015003a006509b100a7
:1009b000110032000a0035006928e100030035000b
:1009c000010028004f01be000000050000004000ab
:1009d000818048008502e900fcff3a0006003700ec
:1009e000f88f4200060035008100d1000080d3005e
:1009f0008502e800fcff3a004f01be00000006003f
:100a00008000eb004f01be00000005000080fb00ed
:100a10008000eb00829fbe00889fbe008a9fbe00c0
:100a2000010578000100e0000400350008003c00ea
:100a30000000e000200032000500370060001000d8
:100a4000e080180002003b0001f024001a0037008b
:100a50000004be006011b8006b0920000982cf00bd
:100a6000020039000882cf000441b0006942520000
:100a70000e00320008003b008281710061016400b9
:100a80008904d1000884d3008b05e8000442e80003
:100a9000f9ff3a00050037000804440089844c003f
:100aa0008b05e9000442e900fbff3a002300070040
:100ab0000af0a70001f0a0004f05be004f04be00e1
:100ac0004f01be00000006000004be000600070043
:100ad0000003be000405be000200be0002000700c5
:100ae000844f750000000600c70ade00f107b2005f
:100af000f50fb20008003200e1cf420002003200e0
:100b00000170a00024000500810f70000100320078
:100b10000408050044000500810f700002003a003f
:100b2000140005008502e9000000400081c0480073
:100b3000fcff3b000170a0002400050081002000a4
:100b4000618055000b003d000b00200061fe2f006e
:100b50000100e1001d003400828171006101640028
:100b60008904d1000884d3000000e800faff3a00ad
:100b7000710020006100640003007000020060004a
:100b80000900320061044400e0844c000988a5009b
:100b9000050032008b05e8006808e10002003a0019
:100ba0008904d1000884d300f20f20000258e1002c
:100bb00005003d00c75ddd00f907b20089807500c2
:100bc00008007800000006000bf827008b00780072
:100bd000000005000200be006450e1000500360080
:100be0006420e100020036000968a30001003a0019
:100bf0000800be000160a0004f06be004f05be0009
:100c00004f04be004f03be0000000600f0ff2f009f
:100c1000f1ff2700f8ff37000020ef000220ef006f
:100c2000c088a900004006000f002100b02e21005e
:100c300000018800000000000000eb0000077800c1
:100c40000c000900002f78000007eb005420ef0093
:100c50000e2eef001e2eef000000eb00a121210060
:100c6000e51d09008018780010cea90010cea9005b
:100c700014cea90010aea90010aea90014aea900b0
:100c8000108ea90040a7a900a1002000f3fd0700d5
:100c9000e0022000303a880044e7a90044c7a900d8
:100ca0004407a9004427a9004447a9004467a900b4
:100cb0004487a900300020000600fc0031742000a9
:100cc00082072000a309200082487800834878002a
:100cd00080487800113a8000618070000600fc00b6
:100ce00021742000620420007305200082487800ef
:100cf00083487800804878004427ef00e002200015
:100d0000303a8800300020000d00fc0031742000d3
:100d100082072000a30920008248780083487800d9
:100d20008048780000002000217420006204200028
:100d30007305200082487800834878008048780056
:100d400042a7ae00feff3700813e2000c3fd070032
:100d500010c0b30086e6b70090c2b300c4e6b70087
:100d6000000220000070880000702500807088005c
:100d700010eea9004188a80041a8a80041c8a90018
:100d800004a1a9000481a90005e1a8000068a90048
:100d90001061a8001021a90011e1a80011a1a9006b
:100da00010a1a8001081a8000821ef000621ef0083
:100db0000ca1ef000ea1ef004408a8004428a900f0
:100dc0004448a9000108a9002108a8001fe1a800c3
:100dd0001fa1a9001ec1a9001ea1a9001e81a90072
:100de0001e61a9001e21a9004d88a9004da8a800d8
:100df0004dc8a8000368a90021e1a80021a1a9000d
:100e000020c1a90020a1a9002081a9002021a900ba
:100e10004e08a9004e28a8004e48a8000388a90043
:100e20002002a9002022a9002042a90020a2a90096
:100e30002062a9002082a90020e2a9002102a900c5
:100e40002122a900700720004011880022a2a900d9
:100e500022c2a90022e2a90021e2a8002182a90061
:100e60004588a90045a8a80045c8a8002168a80091
:100e70002828a80023e2a90023e2a9002342a80011
:100e80002362a9000188a9002188a8004608a800bb
:100e90004628a8004648a9002bc8a9002be8a900ad
:100ea0002c08a9000bc8a9000be8a9000c08a90090
:100eb00001eca90001aca900016ca900014ca9003a
:100ec000012ca900010ca90000eca900008ca900cc
:100ed00000aca90000cca900000ca900002ca900be
:100ee000004ca900006ca900202cef00402cef0062
:100ef000602cef00f01f200020608800020ca90089
:100f0000022ca900024ca900262cef00462cef0071
:100f1000662cef00282cef00482cef00682cef0027
:100f20000aacef0023eca80023cca90043eca800f6
:100f300043cca90063eca80063cca900dabc2a006a
:100f40001b32240030002c00fa608800fb6088000f
:100f500020618800dabc2a001b322400000028002f
:100f6000fa608800fb60880010618800dabc2a0003
:100f70001b32240030002c00fa608800fb608800df
:100f800020628800dabc2a001b32240000002800fe
:100f9000fa608800fb60880010628800dabc2a00d2
:100fa0001b32240030002c00fa608800fb608800af
:100fb00020638800dabc2a001b32240000002800cd
:100fc000fa608800fb6088001063880011eea900b9
:100fd00011aea900116ea900a70037003f0037002d
:100fe00000202000006188000020200000628800ae
:100ff0000020200000638800020ca900022ca80039
:10100000024ca80004acef0028acef0048acef00a5
:1010100068acef00262cef00462cef00662cef00aa
:101020000aacef0023eca80023cca90043eca800f5
:1010300043cca90063eca80063cca900dabc2a0069
:101040001b32240030002c00fa608800fb6088000e
:1010500020618800dabc2a001b322400000028002e
:10106000fa608800fb60880010618800dabc2a0002
:101070001b32240030002c00fa608800fb608800de
:1010800020628800dabc2a001b32240000002800fd
:10109000fa608800fb60880010628800dabc2a00d1
:1010a0001b32240030002c00fa608800fb608800ae
:1010b00020638800dabc2a001b32240000002800cc
:1010c000fa608800fb6088001063880011eea900b8
:1010d00011aea900116ea900670037003500370076
:1010e00000102000006188000010200000628800cd
:1010f0000010200000638800020ca900022ca80048
:10110000024ca8000a2cef0004acef00282cef00e2
:101110005055250040628800a0aa2a00406388003c
:10112000dabc2a001b32240030002c00fa60880050
:10113000fb60880020618800dabc2a001b32240092
:1011400000002c00fa608800fb60880010618800b5
:10115000dabc2a001b32240030002c00fa60880020
:10116000fb60880020628800dabc2a001b32240061
:1011700000002c00fa608800fb6088001062880084
:10118000dabc2a001b32240030002c00fa608800f0
:10119000fb60880020638800dabc2a001b32240030
:1011a00000002c00fa608800fb6088001063880053
:1011b0003100370030003700001020000061880047
:1011c0000010200000628800020ca900022ca80078
:1011d000024ca8000a2cef0004acef00282cef0012
:1011e0000000240040628800dabc2a001b32240080
:1011f00030002c00fa608800fb60880020618800c5
:10120000dabc2a001b32240000002c00fa6088009f
:10121000fb60880010618800dabc2a001b322400c1
:1012200030002c00fa608800fb6088002062880093
:10123000dabc2a001b32240000002c00fa6088006f
:10124000fb60880010628800dabc2a001b32240090
:1012500030002c00fa608800fb6088002063880062
:10126000dabc2a001b32240000002c00fa6088003f
:10127000fb60880010638800218ca900418ca900c4
:10128000618ca900216ca900416ca900616ca900c6
:10129000214ca900414ca900614ca90020eca800f8
:1012a00040eca80060eca8003e2cef005e2cef00a4
:1012b0007e2cef0001eca8000000eb00414e210065
:1012c000ff00090080587800bf72ef00c072ef0085
:1012d000a232ef00a432ef000000eb00415e2100db
:1012e0000801090080587800c172ef00c272ef0057
:1012f0000080eb00814d2100050009008018780076
:101300004832ef004a32ef004c32ef00d472ef0067
:10131000260b0700ee0a07003d0b07005032ef00d6
:1013200010a48000e090880020a480001c12b5006a
:10133000e090880020a480001091880030a48000f4
:101340002212b5001c12b4004200de007092880028
:101350005232ef005432ef005632ef0037013700bf
:10136000ff3ffc004200f8003600f8004400f8009f
:101370008e1f78000e0020000d000900be1f7800af
:101380003200f8000100fc000068a9000021ef0015
:1013900013eeaf000400370090948000100888001e
:1013a00015eea80004003700009580009412b500e7
:1013b0001008880015eea900ff3ffc003200f9007c
:1013c000ae0120000d0009004f1778004f0778008c
:1013d0004400f9003600f9004200f9000100fc0069
:1013e00000400600ff3ffc004200f8003600f80015
:1013f0004400f8008e1f78000e0020000d00090048
:10140000be1f78003200f8000100fc000108a900ae
:101410000821ef000621ef000080eb00814d210044
:101420000500090080187800d2f2ef00a232ef0028
:10143000a432ef00a5f2a900d572ef00d672ef003a
:10144000d772ef00ff3ffc003200f900ae01200030
:101450000d0009004f1778004f0778004400f9008d
:101460003600f9004200f9000100fc0000400600cf
:10147000ff3ffc004200f8003600f8004400f8008e
:101480008e1f78000e0020000d000900be1f78009e
:101490003200f8000100fc000368a9001421ef00ed
:1014a00013aeaf0004003700b0948000d00888006d
:1014b00015aea80004003700009580009812b50012
:1014c000d008880015aea900ff3ffc003200f900eb
:1014d000ae0120000d0009004f1778004f0778007b
:1014e0004400f9003600f9004200f9000100fc0058
:1014f00000400600ff3ffc004200f8003600f80004
:101500004400f8008e1f78000e0020000d00090036
:10151000be1f78003200f8000100fc000388a9001b
:101520001821ef00136eaf0004003700d094800044
:10153000e0088800156ea8000400370000958000c0
:101540009c12b500e0088800156ea900ff3ffc0062
:101550003200f900ae0120000d0009004f1778009d
:101560004f0778004400f9003600f9004200f90006
:101570000100fc0000400600ff3ffc004200f800b4
:101580003600f8004400f8008e1f78000e0020009e
:101590000d000900be1f78003200f8000100fc00b9
:1015a0000168a900bf72ec00bfd2bf008080fb00c1
:1015b00030118000424e210080707900ff3ffc0016
:1015c0003200f900ae0120000d0009004f1778002d
:1015d0004f0778004400f9003600f9004200f90096
:1015e0000100fc0000400600ff3ffc004200f80044
:1015f0003600f8004400f8008e1f78000e0020002e
:101600000d000900be1f78003200f8000100fc0048
:101610000828a9002242ae00000037002222af00b5
:101620002222a900ff3ffc003200f900ae01200099
:101630000d0009004f1778004f0778004400f900ab
:101640003600f9004200f9000100fc0000400600ed
:10165000ff3ffc004200f8003600f8004400f800ac
:101660008e1f78000e0020000d000900be1f7800bc
:101670003200f8000100fc000188a900ff3ffc00d7
:101680003200f900ae0120000d0009004f1778006c
:101690004f0778004400f9003600f9004200f900d5
:1016a0000100fc0000400600ff3ffc004200f80083
:1016b0003600f8004400f8008e1f78000e0020006d
:1016c0000d000900be1f78003200f8000100fc0088
:1016d00001a8a900ff3ffc003200f900ae01200084
:1016e0000d0009004f1778004f0778004400f900fb
:1016f0003600f9004200f9000100fc00004006003d
:10170000ff3ffc004200f8003600f8004400f800fb
:101710008e1f78000e0020000d000900be1f78000b
:101720003200f8000100fc000bc8a900ff3ffc00dc
:101730003200f900ae0120000d0009004f177800bb
:101740004f0778004400f9003600f9004200f90024
:101750000100fc0000400600ff3ffc004200f800d2
:101760003600f8004400f8008e1f78000e002000bc
:101770000d000900be1f78003200f8000100fc00d7
:101780000be8a900ff3ffc003200f900ae01200089
:101790000d0009004f1778004f0778004400f9004a
:1017a0003600f9004200f9000100fc00004006008c
:1017b000ff3ffc004200f8003600f8004400f8004b
:1017c0008e1f78000e0020000d000900be1f78005b
:1017d0003200f8000100fc000c08a900ff3ffc00eb
:1017e0003200f900ae0120000d0009004f1778000b
:1017f0004f0778004400f9003600f9004200f90074
:101800000100fc0000400600c0d2bf00bf52e30050
:1018100007003200c072ec00c0d2bf000080fb00a5
:10182000414e210060c07800c3f2b70001003700cc
:10183000c3f2ef0000000600000006003008800040
:10184000109588004008800020958800eeff070072
:10185000c0ccb300c352b50006003900e0cfb300de
:10186000c352b5000100390001003700c472ef0017
:101870004f043700c3f2ae0028003700c472ef00f7
:10188000b0c8b300c352e30005003a00c3d2bf00a2
:10189000c4f2b700c5f2ef00c6f2ef001e00370039
:1018a000b0c9b300c352e30005003a00c3d2bf0081
:1018b000c4f2b700c7f2ef00c8f2ef00160037001d
:1018c000b0cab300c352e30005003a00c3d2bf0060
:1018d000c4f2b700c9f2ef00caf2ef000e00370001
:1018e000b0cbb300c352e30005003a00c3d2bf003f
:1018f000c4f2b700cbf2ef00ccf2ef0006003700e5
:10190000b0ccb300c352e30003003a00c3d2bf001f
:10191000c4f2b700cdf2ef0025043700c452e20054
:1019200002003a002204370021043700b0c8b30097
:10193000c452e300f4003a0000e0ef00c552e300b7
:1019400003003a00c3d2bf00c5f2b700ed00370074
:10195000c3d2bf00c6f2b70050c5b300c552e30002
:1019600023003a00d572ef00d412a900c652e2005b
:1019700002003600c652d40065f2b7006412e200dd
:1019800013003600d5d2a8006212ec00e090880067
:1019900020938000e29080000200e000020032000c
:1019a000110009000280d800009488000094800093
:1019b000129580002395800000004100e0804900de
:1019c0000001be00c2a68800d3a68800060037002a
:1019d000d8b4ef00dab4ef00262cef002068a9009d
:1019e0000068a90015eea900d312a800c4003700b2
:1019f00060c5b300c552e30023003a00d672ef0081
:101a0000d432a900c652e20002003600c652d40009
:101a10006ff2b7006e12e20013003600d6d2a800b3
:101a20006c12ec00e090880070938000e2908000df
:101a30000200e00002003200110009000280d8001c
:101a40004094880040948000129580002395800087
:101a500000004100e08049000001be00e2a68800cd
:101a6000f3a6880006003700dcb4ef00deb4ef0018
:101a7000462cef002368a9000368a90015aea90051
:101a8000d312a8009e00370070c5b300c552e30012
:101a900023003a00d772ef00d452a900c652e200e8
:101aa00002003600c652d40079f2b7007812e20084
:101ab00013003600d7d2a8007612ec00e090880020
:101ac000c0938000e29080000200e000020032003b
:101ad000110009000280d800809488008094800062
:101ae000129580002395800000004100e0804900ad
:101af0000001be0002a7880013a788000600370077
:101b0000e0b4ef00e2b4ef00662cef002388a900f8
:101b10000388a900156ea900d312a8007800370029
:101b2000c5d2bf0080407800eecf500003003a00dd
:101b300010aea90014aea9007100370010c6b300a2
:101b4000c552e30023003a00d572ef00d412a90079
:101b5000c652e20002003600c652d40065f2b70059
:101b60006412e20013003600d5d2a8006212ec0025
:101b7000e090880020938000e29080000200e00066
:101b800002003200110009000280d8000094880091
:101b90000094800012958000239580000000410091
:101ba000e08049000001be00c2a68800d3a68800dc
:101bb00006003700d8b4ef00dab4ef00262cef00af
:101bc0002068a9000068a90015eea900d312a8009a
:101bd0004b00370020c6b300c552e30023003a0093
:101be000d672ef00d432a900c652e20002003600dd
:101bf000c652d4006ff2b7006e12e2001300360036
:101c0000d6d2a8006c12ec00e0908800709380009f
:101c1000e29080000200e0000200320011000900a2
:101c20000280d80040948800409480001295800083
:101c30002395800000004100e08049000001be00c3
:101c4000e2a68800f3a6880006003700dcb4ef00a7
:101c5000deb4ef00462cef002368a9000368a9005a
:101c600015aea900d312a8002500370030c6b30076
:101c7000c552e30022003a00d772ef00d452a90007
:101c8000c652e20002003600c652d40079f2b70014
:101c90007812e20013003600d7d2a8007612ec00ca
:101ca000e0908800c0938000e29080000200e00095
:101cb00002003200110009000280d80080948800e0
:101cc00080948000129580002395800000004100e0
:101cd000e08049000001be0002a7880013a7880029
:101ce00006003700e0b4ef00e2b4ef00662cef002e
:101cf0002388a9000388a900156ea900d312a800a3
:101d0000c5f2ef002a033700b0c9b300c452e300a4
:101d100070023a0000e0ef00c752e30003003a000f
:101d2000c3d2bf00c7f2b70069023700c3d2bf00f9
:101d3000c8f2b700c852e200df003a0050c5b30055
:101d4000c752e3001f003a00d572ef00d412a90079
:101d50006412e20013003600d5d2a8006212ec0033
:101d6000e090880020938000e29080000200e00074
:101d700002003200110009000280d800009488009f
:101d8000009480001295800023958000000041009f
:101d9000e08049000001be00c2a68800d3a68800ea
:101da00006003700d8b4ef00dab4ef00262cef00bd
:101db0002068a9000068a90015eea900d312a800a8
:101dc000bc00370060c5b300c752e3001f003a00f3
:101dd000d672ef00d432a9006e12e2001300360072
:101de000d6d2a8006c12ec00e090880070938000be
:101df000e29080000200e0000200320011000900c1
:101e00000280d800409488004094800012958000a1
:101e10002395800000004100e08049000001be00e1
:101e2000e2a68800f3a6880006003700dcb4ef00c5
:101e3000deb4ef00462cef002368a9000368a90078
:101e400015aea900d312a8009a00370070c5b300e0
:101e5000c752e3001f003a00d772ef00d452a90026
:101e60007812e20013003600d7d2a8007612ec00f8
:101e7000e0908800c0938000e29080000200e000c3
:101e800002003200110009000280d800809488000e
:101e9000809480001295800023958000000041000e
:101ea000e08049000001be0002a7880013a7880057
:101eb00006003700e0b4ef00e2b4ef00662cef005c
:101ec0002388a9000388a900156ea900d312a800d1
:101ed00078003700c7d2bf0080407800eecf5000b6
:101ee00003003a0010aea90014aea900710037003b
:101ef00010c6b300c752e30023003a00d572ef00ca
:101f0000d412a900c652e20002003600c652d40024
:101f100065f2b7006412e20013003600d5d2a800c3
:101f20006212ec00e090880020938000e290800034
:101f30000200e00002003200110009000280d80017
:101f40000094880000948000129580002395800002
:101f500000004100e08049000001be00c2a68800e8
:101f6000d3a6880006003700d8b4ef00dab4ef003b
:101f7000262cef002068a9000068a90015eea90032
:101f8000d312a8004b00370020c6b300c752e300ad
:101f900023003a00d672ef00d432a900c652e20004
:101fa00002003600c652d4006ff2b7006e12e20093
:101fb00013003600d6d2a8006c12ec00e090880026
:101fc00070938000e29080000200e0000200320086
:101fd000110009000280d8004094880040948000dd
:101fe000129580002395800000004100e0804900a8
:101ff0000001be00e2a68800f3a6880006003700b4
:10200000dcb4ef00deb4ef00462cef002368a9003b
:102010000368a90015aea900d312a8002500370057
:1020200030c6b300c752e30022003a00d772ef0077
:10203000d452a900c652e20002003600c652d400b3
:1020400079f2b7007812e20013003600d7d2a80068
:102050007612ec00e0908800c0938000e29080004f
:102060000200e00002003200110009000280d800e6
:1020700080948800809480001295800023958000d1
:1020800000004100e08049000001be0002a7880076
:1020900013a7880006003700e0b4ef00e2b4ef00b9
:1020a000662cef002388a9000388a900156ea900fb
:1020b000d312a8008601370050c5b300c752e30011
:1020c0003d003a00c8d2bf000080fb00f0928800bb
:1020d000d572ef002068a90015eea9005232ef007a
:1020e00010a48000d0908800409280001a12b500a1
:1020f0001092880072958000839580001092800075
:1021000043fa0700c8f9070021fa070090948800f5
:10211000909480004212b500a09488000068a90045
:102120002068a800262cef00d512a800e0928000bd
:10213000f29280000200e00002003200110009006b
:102140000280d800e0938800f19280001093800014
:10215000808f50000d003200109380005e12b50099
:1021600001e0af000020ee00109188000093800095
:10217000129180000200e00002003200110009000c
:102180000280d800f0938800010037007e32ef0013
:10219000e0938000129580002395800000004100ac
:1021a000e08049000001be00c2a68800d3a68800d6
:1021b000d312a8004501370060c5b300c752e30041
:1021c0003d003a00c8d2bf000080fb004093880069
:1021d000d672ef002368a90015aea9005432ef00b3
:1021e00020a48000d0908800509280001a12b50080
:1021f0002092880092958000a39580002092800014
:1022000003fa070088f90700e1f90700b094880095
:10221000b09480004412b500c09488000368a900ff
:102220002368a800462cef00d612a8003093800047
:10223000429380000200e000020032001100090019
:102240000280d80020948800419380006093800031
:10225000808f50000d003200609380006812b5003e
:1022600001e0af000020ee00109188003093800064
:10227000129180000200e00002003200110009000b
:102280000280d80030948800010037008632ef00c9
:10229000209480001295800023958000000041006a
:1022a000e08049000001be00e2a68800f3a6880095
:1022b000d312a8000501370070c5b300c752e30070
:1022c0003d003a00c8d2bf000080fb009093880018
:1022d000d772ef002388a900156ea9005632ef00cf
:1022e00030a48000d0908800609280001a12b5005f
:1022f00030928800b2958000c395800030928000b3
:10230000c3f9070048f90700a1f90700d094880035
:10231000d09480004612b500e09488000388a9009c
:102320002388a800662cef00d712a80080938000b5
:10233000929380000200e0000200320011000900c8
:102340000280d8006094880091938000b093800050
:10235000808f50000d003200b09380007212b500e3
:1023600001e0af000020ee00109188008093800013
:10237000129180000200e00002003200110009000a
:102380000280d80070948800010037008e32ef0080
:102390006094800012958000239580000000410029
:1023a000e08049000001be0002a7880013a7880052
:1023b000d312a800c5003700c7d2bf008040780004
:1023c000eecf500002003a0014aea800bf00370064
:1023d00010c6b300c752e3003d003a00c8d2bf00a8
:1023e0000080fb00f0928800d572ef002068a90001
:1023f00015eea9005232ef00d0a48000d0908800e2
:10240000409280001a12b5001092880072958000e8
:1024100083958000109280007df9070002f9070083
:102420005bf9070090948800909480004212b500f8
:10243000a09488000068a9002068a800262cef005e
:10244000d512a800e0928000f29280000200e00025
:1024500002003200110009000280d800e0938800d9
:10246000f192800010938000808f50000d003200a8
:10247000109380005e12b50001e0af000020ee0076
:102480001091880000938000129180000200e0000b
:1024900002003200110009000280d800f093880089
:1024a000010037007e32ef00e0938000129580003b
:1024b0002395800000004100e08049000001be003b
:1024c000c2a68800d3a68800d312a8007f003700d8
:1024d00020c6b300c752e3003d003a00c8d2bf0097
:1024e0000080fb0040938800d672ef002368a900ab
:1024f00015aea9005432ef00e0a48000d09088000f
:10250000509280001a12b5002092880092958000a7
:10251000a3958000209280003df90700c2f80700d3
:102520001bf90700b0948800b09480004412b500f5
:10253000c09488000368a9002368a800462cef0017
:10254000d612a80030938000429380000200e00081
:1025500002003200110009000280d8002094880097
:102560004193800060938000808f50000d00320006
:10257000609380006812b50001e0af000020ee001b
:102580001091880030938000129180000200e000da
:1025900002003200110009000280d8003094880047
:1025a000010037008632ef002094800012958000f1
:1025b0002395800000004100e08049000001be003a
:1025c000e2a68800f3a68800d312a8003f003700d7
:1025d00030c6b300c752e3003c003a00c8d2bf0087
:1025e0000080fb0090938800d772ef002388a90039
:1025f000156ea9005632ef00f0a48000d09088003c
:10260000609280001a12b50030928800b295800066
:10261000c395800030928000fdf8070082f8070023
:10262000dbf80700d0948800d09480004612b500f3
:10263000e09488000388a9002388a800662cef0096
:10264000d712a80080938000929380000200e000df
:1026500002003200110009000280d8006094880056
:1026600091938000b0938000808f50000d00320065
:10267000b09380007212b50001e0af000020ee00c0
:102680001091880080938000129180000200e00089
:1026900002003200110009000280d8007094880006
:1026a000010037008e32ef006094800012958000a8
:1026b0002395800000004100e08049000001be0039
:1026c00002a7880013a78800d312a800c7f2ef0062
:1026d000b7003700b0cab300c452e30087003a0025
:1026e00000e0ef00c952e30003003a00c3d2bf008c
:1026f000c9f2b70080003700c352ec00caf2b7003d
:1027000050c5b300c952e30012003a000200200095
:1027100003382400cad2bf00bcf80700fff7070047
:10272000709588008195880072958000839580005f
:1027300010928000b6f807003bf8070094f80700f5
:1027400090948800909480004212b500a094880074
:102750006800370060c5b300c952e30012003a00b8
:102760000200200003382400cad2bf00a7f80700e7
:10277000eaf7070090958800a1958800929580005f
:10278000a395800020928000a1f8070026f807009a
:102790007ff80700b0948800b09480004412b50020
:1027a000c09488005300370070c5b300c952e300dd
:1027b00012003a000200200003382400cad2bf00f1
:1027c00092f80700d5f70700b0958800c1958800fa
:1027d000b2958000c3958000309280008cf807008d
:1027e00011f807006af80700d0948800d0948000a0
:1027f0004612b500e09488003e00370010c6b300d2
:10280000c952e30012003a000200200003382400fd
:10281000cad2bf007df80700c0f707007095880096
:1028200081958800729580008395800010928000c9
:1028300077f80700fcf7070055f807009094880028
:10284000909480004212b500a094880029003700bf
:1028500020c6b300c952e30012003a000200200073
:1028600003382400cad2bf0068f80700abf707009e
:1028700090958800a195880092958000a39580008e
:102880002092800062f80700e7f7070040f8070091
:10289000b0948800b09480004412b500c0948800c1
:1028a0001400370030c6b300c952e30011003a00eb
:1028b0000200200003382400cad2bf0053f80700ea
:1028c00096f70700b0958800c1958800b295800002
:1028d000c3958000309280004df80700d2f70700c2
:1028e0002bf80700d0948800d09480004612b500e1
:1028f000e0948800c9f2ef002d003700b0cbb300a0
:10290000c452e3000a003a0000e0ef00cb52e300bb
:1029100003003a00c3d2bf00cbf2b7000300370078
:10292000c3d2bf00ccf2b700e60307002000370097
:10293000b0ccb300c452e30007003a0000e0ef005f
:10294000cd52e30003003a00c3d2bf00cdf2b7007e
:10295000d203070016003700b0cdb300c452e30025
:1029600007003a0000e0ef00ce52e30003003a0017
:10297000c3d2bf00cef2b700d00307000c0037006f
:10298000b0ceb300c452e30009003a0000e0ef000b
:10299000cf52e30003003a00c3d2bf00cff2b7002a
:1029a00003003700c3d2bf00d0f2b700c003070056
:1029b000d312af001903070030c0b300d252b500e4
:1029c000fa02310012958000239580005095800016
:1029d00061958000800f5100818f5900e802390015
:1029e000adf2a800d252e200f3003a00d5d2bf0007
:1029f00080407800e1cf50000d003a007a32ef00bd
:102a0000d412a90020c0b300d5f2b700e093800033
:102a1000129580002395800000004100e08049006d
:102a20000001be00c2a68800d3a68800e1003700de
:102a3000d5d2bf0080407800e2cf500059003a0064
:102a4000d1938000f0928000808f500016003100fa
:102a50007a32ec00d293800002014100802d2100e7
:102a600060007900d0908800d2958000e3958000c6
:102a7000d0908000e6f707006bf70700c4f7070067
:102a800030618800e09380001295800023958000db
:102a900000004100e08049000001be00c2a688009d
:102aa000d3a688003e003700d572ef00f192800077
:102ab00010938000808f500006003a00d8b4ef00d9
:102ac000dab4ef0010938000d0938800d412a800ed
:102ad0003300370010938000f1928000808f500007
:102ae00018003600d552a800f0928000d0938800dc
:102af000d293800002014100802d21006000790006
:102b0000d0908800d2958000e3958000d09080001e
:102b1000bff7070044f707009df707003061880002
:102b2000f093800012958000239580000000410002
:102b3000e08049000001be00c2a68800d3a688003c
:102b400017003700d572a800f0928000d09388005b
:102b5000d293800002014100802d210060007900a5
:102b6000d0908800d2958000e3958000d0908000be
:102b7000a7f707002cf7070085f7070030618800ea
:102b8000f0938000129580002395800000004100a2
:102b9000e08049000001be00c2a68800d3a68800dc
:102ba00084003700d5d2bf0080407800e4cf5000c9
:102bb0001e003a007a32ed00d293800002014100fb
:102bc000802d210060007900d0908800d29580008f
:102bd000e3958000d09080008df7070012f7070082
:102be0006bf7070030618800f09380001295800039
:102bf0002395800000004100e08049000001be00f4
:102c0000c2a68800d3a68800d193800010938000cc
:102c1000808f500004003a00d572ef00d8b4ef0066
:102c2000dab4ef00d412a80062003700d5d2bf009a
:102c300080407800e8cf50001e003a007a32ec0065
:102c4000d293800002014100802d210060007900b4
:102c5000d0908800d2958000e3958000d0908000cd
:102c60006bf70700f0f6070049f7070030618800ae
:102c7000f0938000129580002395800000004100b1
:102c8000e08049000001be00c2a68800d3a68800eb
:102c9000d193800010938000808f500004003a0090
:102ca000d572ef00d8b4ef00dab4ef00d412a80068
:102cb0004000370000c4b300d552e3001a003a00c8
:102cc00010938000d0938800d293800002014100cd
:102cd000802d210060007900d0908800d29580007e
:102ce000e3958000d090800049f70700cef60700fa
:102cf00027f707003061880000c8b300d5f2b7009d
:102d0000009480001295800023958000000041000f
:102d1000e08049000001be00c2a68800d3a688005a
:102d2000d412a9002300370000c8b300d552e30035
:102d300020003a007a12e200160036007a32ed00e6
:102d4000d293800002014100802d210060007900b3
:102d5000d0908800d2958000e3958000d0908000cc
:102d60002bf70700b0f6070009f70700306188006d
:102d7000009480001295800023958000000041009f
:102d8000e08049000001be00c2a68800d3a68800ea
:102d900008003700d572ef00262cef000021ef006d
:102da0002068a9000068a90015eea900d8b4ef00ba
:102db000dab4ef00f1013700d2d2bf0080407800d2
:102dc000e1cf5000f5003a00d6d2bf008040780035
:102dd000e1cf50000d003a008232ef00d432a9005a
:102de00020c0b300d6f2b700209480001295800076
:102df0002395800000004100e08049000001be00f2
:102e0000e2a68800f3a68800e3003700d6d2bf0010
:102e100080407800e2cf500059003a0011948000c1
:102e200040938000808f5000160031008232ec0009
:102e30001294800002014100802d21006000790081
:102e4000d0908800d2958000e3958000d0908000db
:102e5000eff6070074f60700cdf607003062880031
:102e6000209480001295800023958000000041008e
:102e7000e08049000001be00e2a68800f3a68800b9
:102e80003e003700d672ef004193800060938000cf
:102e9000808f500006003a00d692a800dcb4ef0004
:102ea000deb4ef006093800010948800d432a80054
:102eb0006093800041938000808f5000180036009e
:102ec000d652a8004093800010948800129480008d
:102ed00002014100802d210060007900d09088001f
:102ee000d2958000e3958000d0908000c8f607005e
:102ef0004df60700a6f60700306288003094800087
:102f0000129580002395800000004100e080490078
:102f10000001be00e2a68800f3a688001700370073
:102f2000d672a8004093800010948800129480000c
:102f300002014100802d210060007900d0908800be
:102f4000d2958000e3958000d0908000b0f6070015
:102f500035f607008ef60700306288003094800056
:102f6000129580002395800000004100e080490018
:102f70000001be00e2a68800f3a6880086003700a4
:102f8000d6d2bf0080407800e4cf50001f003a0046
:102f90008232ed001294800002014100802d210058
:102fa00060007900d0908800d2958000e395800081
:102fb000d090800096f607001bf6070074f6070015
:102fc0003062880030948000129580002395800044
:102fd00000004100e08049000001be00e2a6880038
:102fe000f3a688001194800060938000808f5000c9
:102ff00005003a00d652a900d692a800dcb4ef0032
:10300000deb4ef00d432a80063003700d6d2bf0090
:1030100080407800e8cf50001f003a008232ec0078
:103020001294800002014100802d2100600079008f
:10303000d0908800d2958000e3958000d0908000e9
:1030400073f60700f8f5070051f6070030628800b4
:10305000309480001295800023958000000041008c
:10306000e08049000001be00e2a68800f3a68800c7
:103070001194800060938000808f500005003a001a
:10308000d672a900d692a800dcb4ef00deb4ef003f
:10309000d432a8004000370000c4b300d652e30089
:1030a0001a003a0060938000109488001294800007
:1030b00002014100802d210060007900d09088003d
:1030c000d2958000e3958000d090800050f60700f4
:1030d000d5f507002ef607003062880000c8b3005f
:1030e000d6f2b700409480001295800023958000ae
:1030f00000004100e08049000001be00e2a6880017
:10310000f3a68800d432a9002300370000c8b3001a
:10311000d652e30020003a008212e2001600360088
:103120008232ed001294800002014100802d2100c6
:1031300060007900d0908800d2958000e3958000ef
:10314000d090800032f60700b7f5070010f60700b0
:1031500030628800409480001295800023958000a2
:1031600000004100e08049000001be00e2a68800a6
:10317000f3a6880008003700d672ef00462cef0057
:103180001421ef002368a9000368a90015aea90067
:10319000dcb4ef00deb4ef00f8003700d2d2bf009d
:1031a00080407800e2cf5000f4003a00d7d2bf0050
:1031b00080407800e1cf50000d003a008a32ef00e5
:1031c000d452a90020c0b300d7f2b70060948000a9
:1031d000129580002395800000004100e0804900a6
:1031e0000001be0002a7880013a78800e300370093
:1031f000d7d2bf0080407800e2cf500059003a009b
:103200005194800090938000808f50001600310010
:103210008a32ec005294800002014100802d21008e
:1032200060007900d0908800d2958000e3958000fe
:10323000d0908000f6f507007bf50700d4f5070075
:103240003063880060948000129580002395800090
:1032500000004100e08049000001be0002a7880094
:1032600013a788003e003700d772ef0091938000cb
:10327000b0938000808f500006003a00d792a800db
:10328000e0b4ef00e2b4ef00d452a800b0938000a5
:1032900050948800b093800091938000808f5000fc
:1032a00018003600d752a8009093800050948800f0
:1032b0005294800002014100802d210060007900bd
:1032c000d0908800d2958000e3958000d090800057
:1032d000cff5070054f50700adf50700306388000f
:1032e00070948000129580002395800000004100ba
:1032f000e08049000001be0002a7880013a78800f3
:1033000017003700d772a80090938000509488006f
:103310005294800002014100802d2100600079005c
:10332000d0908800d2958000e3958000d0908000f6
:10333000b7f507003cf5070095f5070030638800f6
:103340007094800012958000239580000000410059
:10335000e08049000001be0002a7880013a7880092
:1033600086003700d7d2bf0080407800e4cf5000fd
:103370001f003a008a32ed005294800002014100a1
:10338000802d210060007900d0908800d2958000c7
:10339000e3958000d09080009df5070022f507009e
:1033a0007bf50700306388007094800012958000e0
:1033b0002395800000004100e08049000001be002c
:1033c00002a7880013a7880051948000b093800062
:1033d000808f500005003a00d752a900d792a8006c
:1033e000e0b4ef00e2b4ef00d452a800630037006d
:1033f000d7d2bf0080407800e8cf50001f003a00cd
:103400008a32ec005294800002014100802d21009c
:1034100060007900d0908800d2958000e39580000c
:10342000d09080007af50700fff4070058f50700f8
:10343000306388007094800012958000239580008e
:1034400000004100e08049000001be0002a78800a2
:1034500013a7880051948000b0938000808f5000a3
:1034600005003a00d772a900d792a800e0b4ef0097
:10347000e2b4ef00d452a8004000370000c4b3000b
:10348000d752e3001a003a00b093800050948800ad
:103490005294800002014100802d210060007900db
:1034a000d0908800d2958000e3958000d090800075
:1034b00057f50700dcf4070035f507003063880096
:1034c00000c8b300d7f2b700809480001295800046
:1034d0002395800000004100e08049000001be000b
:1034e00002a7880013a78800d452a9002300370040
:1034f00000c8b300d752e30020003a008a12e2006d
:10350000160036008a32ed0052948000020141001c
:10351000802d210060007900d0908800d295800035
:10352000e3958000d090800039f50700bef40700d5
:1035300017f50700306388008094800012958000a2
:103540002395800000004100e08049000001be009a
:1035500002a7880013a7880008003700d772ef0081
:10356000662cef001821ef002388a9000388a9002a
:10357000156ea900e0b4ef00e2b4ef0027000700e9
:10358000a5f2ae0008003700a232ef00a432ef002f
:103590000821ef000621ef000080eb00814d2100a3
:1035a00005000900801878000a003700a5f2ae0077
:1035b00008003700a232ef00a432ef000821ef002c
:1035c0000621ef000080eb00814d2100050009007d
:1035d000801878008af30700d0908800f09480006b
:1035e0001a12b60070918800f0948000e090880074
:1035f0001c32d500709180001c12b5000095880027
:10360000128eaa00108ea900a412af0014eea8001a
:10361000a412ae0014eea90088f83700d2f2ef0031
:10362000aab2ef00acb2ef00d172ef00d1d2bf006e
:103630000080fb00c200dd00804d210000804000c2
:103640001000be000001be00509580006195800012
:10365000800f5100818f59000a003100d1d2bf0084
:103660000080fb00c200dd00804d21000080400092
:103670001000be005095880061958800d1d2bf002f
:10368000d2f2b700d172ec00d1d2bf0080407800f6
:10369000e3cf5000e5ff3a00d312a9000000060076
:1036a00050c5b300c952e30012003a0002002000e6
:1036b00003382400cad2bf00d4f4070017f407006f
:1036c00070958800819588007295800083958000b0
:1036d00010928000cef4070053f40700acf407000a
:1036e00090948800909480004212b500a0948800c5
:1036f0006800370060c5b300c952e30012003a0009
:103700000200200003382400cad2bf00bff4070023
:1037100002f4070090958800a1958800929580009a
:10372000a395800020928000b9f407003ef40700c2
:1037300097f40700b0948800b09480004412b5005c
:10374000c09488005300370070c5b300c952e3002d
:1037500012003a000200200003382400cad2bf0041
:10376000aaf40700edf30700b0958800c195880022
:10377000b2958000c395800030928000a4f40700c9
:1037800029f4070082f40700d0948800d0948000c8
:103790004612b500e09488003e00370010c6b30022
:1037a000c952e30012003a0002002000033824004e
:1037b000cad2bf0095f40700d8f3070070958800bf
:1037c000819588007295800083958000109280001a
:1037d0008ff4070014f407006df40700909488003c
:1037e000909480004212b500a09488002900370010
:1037f00020c6b300c952e30012003a0002002000c4
:1038000003382400cad2bf0080f40700c3f30700c6
:1038100090958800a195880092958000a3958000de
:10382000209280007af40700fff3070058f40700a5
:10383000b0948800b09480004412b500c094880011
:103840001400370030c6b300c952e30011003a003b
:103850000200200003382400cad2bf006bf4070026
:10386000aef30700b0958800c1958800b29580003e
:10387000c39580003092800065f40700eaf30700ea
:1038800043f40700d0948800d09480004612b5001d
:10389000e0948800c9f2ef0000000600cd52e2007b
:1038a00001003a008a010700cdf2ef000000060097
:1038b000cff2ef00d0f2ef0000000600cef2ef00f2
:1038c00000000600cbd2bf0080407800e1cf50005e
:1038d00005003a00ccd2bf000080fb004300dd00b1
:1038e000f09488002e013700cbd2bf0080407800d2
:1038f000e7cf50003a003a00ccd2bf000080fb0076
:10390000c0928800c292800002014100802d2100f7
:1039100060007900d092880002002800f33f240064
:10392000d09280003af407007cf30700d09588001d
:10393000e1958800d412ae000c003700129380008d
:1039400002014100802d210060007900d0908800a4
:10395000d2958000e3958000d09080002cf4070081
:10396000b1f307000af4070030618800d432ae00da
:103970000c0037006293800002014100802d21007d
:1039800060007900d0908800d2958000e395800097
:10399000d09080001ef40700a3f30700fcf307009b
:1039a00030628800d452ae000c003700b293800021
:1039b00002014100802d210060007900d090880034
:1039c000d2958000e3958000d090800010f407002d
:1039d00095f30700eef3070030638800f00037002e
:1039e000cbd2bf0080407800efcf500011003a00ea
:1039f000cc72ec000200200003382400ccd2bf00bf
:103a000002f4070045f3070070958800819588004f
:103a1000709580009095880080958000a095880022
:103a200070958000b095880080958000c0958800d2
:103a3000db003700cbd2bf0080407800f0cf5000d1
:103a40000a003a00ccd2bf000080fb00109388002f
:103a5000ccd2bf000080fb0060938800ccd2bf00b6
:103a60000080fb00b0938800cd003700cbd2bf00b0
:103a700080407800f1cf500007003a00ccd2bf0060
:103a80005df2b700e092800030938800e092800001
:103a900080938800c2003700cbd2bf0080407800fe
:103aa000f2cf500007003a00ccd2bf0061f2b7005d
:103ab000009380005093880000938000a0938800ba
:103ac000b7003700cbd2bf0080407800f3cf500062
:103ad00007003a00cc52d40065f2b7002093800072
:103ae0007093880020938000c0938800ac0037005a
:103af000cbd2bf0080407800f5cf500054003a0090
:103b000081928000ccd2bf000080fb00810f50006a
:103b10004e003200cc52e20002003a003c010700a5
:103b200047003700ccd2bf0080407800eccf500077
:103b300002003a009001070041003700ccd2bf00dc
:103b400080407800edcf500002003a00e30107000a
:103b50003b003700ccd2bf0080407800eecf500051
:103b600002003a003602070035003700ccd2bf0011
:103b700080407800efcf500002003a008902070031
:103b80002f003700ccd2bf0080407800f0cf50002b
:103b900002003a00dc02070029003700ccd2bf0047
:103ba00080407800f1cf500002003a002f03070058
:103bb00023003700ccd2bf0080407800f2cf500005
:103bc00002003a00820307001d003700ccd2bf007c
:103bd00080407800f3cf500002003a00d503070080
:103be00017003700ccd2bf0080407800f4cf5000df
:103bf00002003a002804070011003700ccd2bf00b1
:103c000080407800f5cf500002003a007b040700a6
:103c10000b003700ccd2bf0080407800f6cf5000b8
:103c200002003a00ce04070005003700ccd2bf00e6
:103c300080407800f7cf500001003a0021050700ce
:103c4000ccd2bf000080fb00809288005400370077
:103c500020c4b300cb52e3000e003a00cc52e20085
:103c600004003a007100070010cea90014cea9008c
:103c7000070037004c00070010cea90014cea800a2
:103c80000821ef000621ef00a232ef00a432ef007e
:103c900043003700d0c6b300cb52e30012003a0015
:103ca0000200200003302400ccd2bf0057f30700ed
:103cb0009af207000200200003f0230038f2070008
:103cc00030958800419588003295800043958000aa
:103cd000709280004ef30700d3f2070007f307004d
:103ce000409288002e003700e0c6b300cb52e300bc
:103cf00012003a000200200003302400ccd2bf00a2
:103d000042f3070085f207000200200003f02300c1
:103d100023f2070030958800419588003295800095
:103d2000439580007092800039f30700bef20700cf
:103d3000f2f207005092880019003700f0c6b30075
:103d4000cb52e30012003a000200200003302400ae
:103d5000ccd2bf002df3070070f207000200200054
:103d600003f023000ef2070030958800419588008b
:103d700032958000439580007092800024f3070004
:103d8000a9f20700ddf20700609288000400370006
:103d9000b0c7b300cb52e30001003a0002000700b5
:103da000cbf2ef0000000600262cef00462cef00bf
:103db000662cef002068a9002368a9002388a900c9
:103dc00015eea90015aea900156ea900d572ef0079
:103dd000d672ef00d772ef00d472ef00d172ef000d
:103de00020c0b300d152e3000a003e00d1d2bf0090
:103df0000080fb00c200dd00804d210000814000fa
:103e0000f0ff2f00f1ff2f000089be00d172ec00ff
:103e1000f3ff3900d2f2ef00aab2ef00acb2ef002c
:103e200010aea90014aea90000000600d172ef0088
:103e300020c0b300d152e3000a003e00d1d2bf003f
:103e40000080fb00c200dd00804d210000814000a9
:103e5000f0ff2f00f1ff2f000089be00d172ec00af
:103e6000f3ff3900d2f2ef00aab2ef00acb2ef00dc
:103e7000262cef00462cef00662cef002068a900ee
:103e80002368a9002388a90011eea90015eea90056
:103e900011aea90015aea900116ea900156ea900fa
:103ea000d572ef00d672ef00d772ef00d472ef0038
:103eb000070007004832ef004a32ef004c32ef00b3
:103ec0005300070010aea90014aea90000000600c0
:103ed000f0072000c0928800c292800002014100d9
:103ee000802d210060007900d09288000200280017
:103ef000f33f2400d0928000c5f2070007f20700cc
:103f0000d0958800e1958800a0c0b3005df2b700ad
:103f100040c1b30061f2b700600720001093880031
:103f2000a0c0b30065f2b7004832ef0060ec230098
:103f300080958800ae32ef0000042000f0948800e5
:103f4000e0928000309388000093800050938800b6
:103f50001093800060938800209380007093880005
:103f60004a32ef007095800090958800809580001f
:103f7000a0958800e09280008093880000938000e4
:103f8000a093880010938000b09388002093800055
:103f9000c09388004c32ef0070958000b095880087
:103fa00080958000c09588000000060010c0b30016
:103fb000d1f2b700f0c7b300d152e30010003e00c9
:103fc000d1d2bf0091f207003df107000001be0011
:103fd00090c225005123240013f207006cf2070061
:103fe000112d2100914078008180fb0081804000ec
:103ff000822d210080307900d172ec00edff390074
:10400000f01f2000b09e8800d832ef0000000600ac
:1040100080fa2d0000a4880060312d0010a48800d3
:1040200080732c0020a4880060c02b0030a488007e
:1040300040172b0040a48800a0772a0050a48800d5
:10404000f0e0290060a48800c052290070a4880014
:1040500080cc280080a48800d04d280090a488003f
:1040600030d62700a0a4880050652700b0a488009f
:10407000d0fa2600c0a4880040962600d0a488006c
:1040800050372600e0a48800c0dd2500f0a4880099
:104090003089250000a588006039250010a588001a
:1040a00000ee240020a58800f0a6240030a588009a
:1040b000d063240040a588007024240050a5880007
:1040c000b0e8230060a5880040b0230070a58800f8
:1040d000f07a230080a58800b048230090a58800ce
:1040e00030192300a0a5880070ec2200b0a588003c
:1040f00020c22200c0a58800409a2200d0a58800d6
:1041000090742200e0a5880000512200f0a58800ec
:10411000702f220000a68800d00f220010a6880071
:10412000e0f1210020a68800b0d5210030a688004b
:1041300010bb210040a68800e0a1210050a6880005
:10414000308a210060a68800c073210070a6880014
:10415000a05e210080a68800b04a210090a68800b9
:10416000d0372100a0a6880010262100b0a6880024
:10417000d8b3ef000000060080fa2d0000a48800ec
:10418000801a2d0010a48800506c2c0020a48800f8
:1041900040a52b0030a48800d02d2b0040a488001f
:1041a000a07a2a0050a4880050ef290060a488005b
:1041b0000050290070a48800b0ba280080a48800ac
:1041c0002061280090a48800e0c12700a0a48800f6
:1041d00040722700b0a48800d0fa2600c0a488004e
:1041e000d08a2600d0a48800b0332600e0a488003e
:1041f00030d02500f0a488007094250000a5880028
:10420000e03a250010a5880030f5240020a588009c
:1042100090a5240030a58800f05a240040a588000d
:10422000202e240050a5880080de230060a5880091
:10423000b0b6230070a58800f07a230080a588001e
:10424000f042230090a5880070172300a0a58800e5
:10425000a0e52200b0a58800d0c72200c0a5880034
:10426000009b2200d0a5880020782200e0a58800cd
:1042700050502200f0a58800002b220000a68800e4
:10428000a014220010a68800d0ec210020a68800ef
:10429000e0d8210030a6880010bb210040a688008d
:1042a000109f210050a688004089210060a6880048
:1042b0006070210070a688007061210080a68800cf
:1042c000104b210090a68800a0392100a0a68800ec
:1042d000c0252100b0a6880000000600d0122e00e4
:1042e00000a4880060312d0010a48800f05d2c002f
:1042f00020a4880090b92b0030a48800a0fd2a00db
:1043000040a48800f08c2a0050a48800d0e3290043
:1043100060a488004060290070a48800f0c92800cb
:1043200080a48800003d280090a4880070e8270041
:10433000a0a4880020522700b0a48800000727000e
:10434000c0a4880040962600d0a48800902c2600a7
:10435000e0a4880050da2500f0a48800607c2500e5
:1043600000a588000044250010a5880070ef2400f7
:1043700020a58800b0ad240030a58800806224000c
:1043800040a58800101c240050a58800d0f123000f
:1043900060a58800a0a6230070a5880010812300d6
:1043a00080a58800b048230090a58800d013230082
:1043b000a0a58800c0ea2200b0a58800c0bb2200ea
:1043c000c0a58800909f2200d0a5880050752200cb
:1043d000e0a5880060542200f0a58800d02e2200bd
:1043e00000a68800900b220010a6880070f621001d
:1043f00020a68800e0d0210030a6880010be210051
:1044000040a68800e0a1210050a6880080872100f6
:1044100060a68800f072210070a68800705b210001
:1044200080a68800504d210090a6880030382100d9
:10443000a0a68800c0272100b0a6880000000600c2
:1044400090022e0000a4880060482d0010a488006f
:1044500080732c0020a4880000ac2b0030a48800be
:10446000d0102b0040a48800705f2a0050a4880060
:1044700010f5290060a488007055290070a48800f8
:1044800040d9280080a48800604b280090a48800b0
:1044900060c62700a0a4880090762700b0a48800fa
:1044a000b0e82600c0a48800c0a12600d0a48800df
:1044b00050372600e0a4880090d32500f0a488009f
:1044c000f085250000a58800502d250010a5880046
:1044d00010f8240020a5880040a8240030a58800fa
:1044e000306a240040a588004023240050a588009d
:1044f000c0e0230060a58800d0b8230070a5880024
:10450000e071230080a58800704e230090a58800ec
:1045100030192300a0a5880050e72200b0a588002c
:1045200090c02200c0a5880030942200d0a5880049
:10453000a0792200e0a58800b0512200f0a58800f3
:10454000a032220000a68800300f220010a68800aa
:10455000f0ed210020a6880000da210030a68800b6
:1045600080b6210040a68800c0a4210050a6880083
:10457000308a210060a688004071210070a6880062
:10458000d05d210080a68800a047210090a6880069
:10459000603a2100a0a6880060262100b0a688000d
:1045a00000000600001b2e0000a4880000392d002a
:1045b00010a4880040892c0020a4880060c02b0033
:1045c00030a4880000042b0040a4880090712a00c9
:1045d00050a4880020ca290060a48800b065290082
:1045e00070a4880010cf280080a48800e05928001b
:1045f00090a48800f0d32700a0a48800605627006c
:10460000b0a48800100b2700c0a4880020852600d5
:10461000d0a4880030422600e0a48800c0dd250038
:10462000f0a48800907f250000a588005036250062
:1046300010a58800a0e2240020a5880070b0240006
:1046400030a588001065240040a58800802a240039
:1046500050a5880080e7230060a58800c0a823003b
:1046600070a588001083230080a5880020402300c7
:1046700090a58800a01e2300a0a5880070ec220051
:10468000b0a5880050bd2200c0a58800c0982200b7
:10469000d0a58800e06e2200e0a58800c055220069
:1046a000f0a588002030220000a68800d012220049
:1046b00010a6880050f1210020a68800f0d121002a
:1046c00030a6880020bf210040a68800a09d2100c0
:1046d00050a68800e08c210060a68800c0732100ed
:1046e00070a68800405c210080a68800f049210067
:1046f00090a6880000352100a0a68800702821001f
:10470000b0a688000000060040de2d0000a488004e
:1047100010502d0010a48800c07a2c0020a488001e
:10472000d0d42b0030a4880040172b0040a4880070
:1047300080652a0050a4880030db290060a488002e
:10474000303d290070a4880070de280080a4880015
:104750003050280090a48800a0e12700a0a4880081
:1047600030632700b0a48800b0ec2600c0a4880005
:1047700090a52600d0a4880030272600e0a4880059
:1047800000e82500f0a488003089250000a58800f5
:104790005030250010a5880030eb240020a58800ab
:1047a000309c240030a58800c06c240040a58800ff
:1047b000b025240050a5880060ee230060a5880085
:1047c00020af230070a58800e073230080a5880037
:1047d0006050230090a5880020112300a0a5880028
:1047e00090f12200b0a5880020c22200c0a5880058
:1047f000b0952200d0a5880020732200e0a5880093
:10480000a04b2200f0a58800f033220000a688000b
:104810006010220010a68800c0f4210020a68800a5
:1048200020d5210030a6880080b7210040a688004e
:10483000c0a5210050a688002086210060a688001f
:104840005076210070a68800a05e210080a6880016
:104850007048210090a6880020372100a0a688007b
:1048600060232100b0a688000000060070f62d002d
:1048700000a48800c0162d0010a4880080902c0091
:1048800020a4880030c72b0030a48800902a2b0079
:1048900040a48800a0772a0050a48800d0cf290027
:1048a00060a48800504d290070a4880030b828000a
:1048b00080a48800b05e280090a4880080d82700db
:1048c000a0a4880010702700b0a48800c0f82600bb
:1048d000c0a48800f0882600d0a48800d045260017
:1048e000e0a4880080ce2500f0a48800d0922500a6
:1048f00000a588006039250010a5880070e5240017
:1049000020a5880040a4240030a58800a0592400d8
:1049100040a58800f02c240050a58800d0e9230091
:1049200060a58800a0b5230070a58800f079230059
:1049300080a588000042230090a5880070202300f5
:10494000a0a58800d0e42200b0a5880000c72200fe
:10495000c0a58800409a2200d0a58800507022008f
:10496000e0a58800b04f2200f0a58800602a220050
:1049700000a688000014220010a6880070f2210012
:1049800020a6880060d8210030a6880080ba2100c7
:1049900040a68800909e210050a68800d08d21005e
:1049a00060a68800f06f210070a6880010612100c9
:1049b00080a68800b04a210090a68800b03521006a
:1049c000a0a6880060252100b0a68800000006008f
:1049d00050e62d0000a48800902d2d0010a4880022
:1049e000605a2c0020a48800b0db2b0030a4880083
:1049f000b01d2b0040a48800e0892a0050a4880044
:104a0000f0e0290060a488009042290070a488008a
:104a100060c7280080a48800a03a280090a48800dd
:104a200030e62700a0a4880080672700b0a4880093
:104a3000f0042700c0a4880050942600d0a4880069
:104a4000c02a2600e0a4880060eb2500f0a48800be
:104a5000d07a250000a588008042250010a5880096
:104a600000ee240020a58800d09e240030a58800f8
:104a70004061240040a58800e01a240050a5880069
:104a8000a0f0230060a5880050b1230070a5880025
:104a90000080230080a58800c047230090a58800df
:104aa000f0122300a0a5880040f32200b0a58800e2
:104ab000f0ba2200c0a58800d09e2200d0a58800b0
:104ac00090742200e0a58800004d2200f0a5880027
:104ad000302e220000a68800000b220010a68800bd
:104ae000e0f5210020a6880030d6210030a68800fd
:104af00090bd210040a6880070a1210050a688002a
:104b00000087210060a688003077210070a6880009
:104b1000105b210080a68800f04c210090a6880040
:104b2000d0372100a0a6880010242100b0a688005c
:104b30000000060080fe2d0000a48800501e2d00fd
:104b400010a48800f06f2c0020a48800a0a82b00df
:104b500030a4880010312b0040a48800b07d2a00ca
:104b600050a4880030f2290060a48800c0522900b7
:104b700070a4880040bd280080a488000049280057
:104b800090a4880020c42700a0a488006074270097
:104b9000b0a48800d0fc2600c0a48800d09f2600c6
:104ba000d0a4880080352600e0a48800e0d125004c
:104bb000f0a488001096250000a58800d02b2500c1
:104bc00010a58800a0f6240020a58800f0a62400e7
:104bd00030a58800305c240040a588001022240005
:104be00050a58800a0df230060a58800c0b723007f
:104bf00070a58800f07b230080a58800704d2300fd
:104c000090a5880050182300a0a5880080e6220007
:104c1000b0a58800a0c82200c0a58800709322001b
:104c2000d0a58800e0782200e0a58800005122008d
:104c3000f0a58800a02b220000a68800900e22007c
:104c400010a6880060ed210020a6880070d9210000
:104c500030a6880090bb210040a6880050a4210007
:104c600050a68800b089210060a68800d07021007d
:104c700070a68800e061210080a6880040472100de
:104c800090a68800003a2100a0a6880010262100e6
:104c9000b0a6880000000600f0162e0000a48800d0
:104ca00030352d0010a4880090612c0020a48800cd
:104cb000f0bc2b0030a48800d0002b0040a488005a
:104cc000f08f2a0050a48800b0e6290060a4880074
:104cd0000063290070a4880080cc280080a488008c
:104ce000603f280090a48800b0d12700a0a48800cd
:104cf00040542700b0a4880000092700c0a4880001
:104d000020982600d0a4880060402600e0a48800f7
:104d100000dc2500f0a48800007e250000a58800a6
:104d20009045250010a5880030e1240020a58800ca
:104d300010af240030a58800d063240040a588006f
:104d4000401d240050a5880060e6230060a588006f
:104d5000b0a7230070a588001082230080a58800da
:104d6000a049230090a58800c01d2300a0a58800ad
:104d700090eb2200b0a5880090bc2200c0a588005e
:104d800050a02200d0a58800306e2200e0a5880047
:104d900010552200f0a58800702f220000a6880080
:104da000300c220010a68800c0f0210020a6880048
:104db00060d1210030a6880090be210040a6880066
:104dc00060a2210050a68800708c210060a6880097
:104dd0005073210070a68800d05b210080a6880057
:104de000b04d210090a68800a0342100a0a6880024
:104df00020282100b0a688000000060040da2d001f
:104e000000a48800304c2d0010a4880020772c00ce
:104e100020a4880060af2b0030a4880000142b0071
:104e200040a4880070622a0050a48800f0f729008e
:104e300060a488002058290070a48800d0db2800d6
:104e400080a48800d04d280090a48800a0c8270026
:104e5000a0a4880010612700b0a48800b0ea260052
:104e6000c0a48800b0a32600d0a488002039260062
:104e7000e0a4880040e62500f0a488009087250083
:104e800000a58800d02e250010a5880080f92400f8
:104e900020a58800d09a240030a58800806b2400cb
:104ea00040a588007024240050a58800e0e123007c
:104eb00060a5880010ae230070a58800e072230072
:104ec00080a58800604f230090a58800201a230049
:104ed000a0a58800b0f02200b0a5880050c1220033
:104ee000c0a58800f0942200d0a58800507a220046
:104ef000e0a58800f04a2200f0a588005033220087
:104f000000a68800d00f220010a6880080ee2100a5
:104f100020a68800a0d4210030a6880000b7210078
:104f200040a6880040a5210050a68800a08a210044
:104f300060a68800e075210070a68800405e210010
:104f400080a688000048210090a68800b03a210081
:104f5000a0a6880010232100b0a68800000006004b
:104f6000101f2e0000a48800f0122d0010a488004d
:104f7000e08c2c0020a48800c0c32b0030a4880043
:104f800030072b0040a4880090742a0050a48800a9
:104f900000cd290060a488007068290070a48800f2
:104fa000a0d1280080a48800405c280090a488003c
:104fb00030d62700a0a4880080582700b0a488001d
:104fc000c0f62600c0a4880000872600d0a4880070
:104fd00000442600e0a4880070df2500f0a48800cb
:104fe0004091250000a58800d037250010a5880035
:104ff00010e4240020a58800c0b1240030a588005a
:105000006058240040a58800b02b240050a58800db
:10501000b0e8230060a58800d0a9230070a588000f
:10502000f078230080a588001041230090a5880017
:10503000901f2300a0a5880040ed2200b0a58800a5
:1050400030c62200c0a5880080992200d0a5880023
:10505000906f2200e0a5880070562200f0a588001d
:10506000c029220000a688006013220010a6880034
:10507000e0f1210020a6880070d2210030a688002f
:1050800000ba210040a68800109e210050a688008a
:10509000508d210060a688003074210070a6880021
:1050a000a060210080a68800504a210090a68800b8
:1050b00060352100a0a68800c0282100b0a6880085
:1050c0000000060040e22d0000a48800f0532d00ef
:1050d00010a48800d0562c0020a4880040d82b00b3
:1050e00030a48800701a2b0040a4880080682a0031
:1050f00050a4880010de290060a48800e03f290049
:1051000070a4880000e1280080a48800a052280034
:1051100090a48800e0e32700a0a488005065270041
:10512000b0a48800b0ee2600c0a4880070922600cb
:10513000d0a48800f0282600e0a48800b0e925006b
:10514000f0a48800c08a250000a58800f040250052
:1051500010a5880090ec240020a58800809d2400e4
:1051600030a58800106e240040a58800b0192400e6
:1051700050a5880080ef230060a5880040b0230080
:1051800070a58800e074230080a58800c046230035
:1051900090a5880010122300a0a5880060f22200cc
:1051a000b0a58800f0c22200c0a58800109e220091
:1051b000d0a58800e0732200e0a58800504c2200b2
:1051c000f0a588009034220000a68800600a220022
:1051d00010a6880050f5210020a68800b0d5210037
:1051e00030a6880000b8210040a68800f0a0210069
:1051f00050a688009086210060a68800c076210015
:1052000070a68800005f210080a68800904c2100d5
:1052100090a6880080372100a0a68800b023210036
:08522000b0a6880000000600a2
:020000040000fa
:105228001a12000014000000800000002e12000076
:105238007400000080000000a21200001c000000a2
:1052480080000000be1200001a000000800000006c
:10525800d81200000002000080000000d8140000ee
:105268000c00000080000000e41400000a020000a6
:085278008000000000000000ae
:00000001FF
